:1038C7000FAA0FA50F9F0F9A0F940F8D0F870F80C9
:1038D7000F780F710F680F600F570F4E0F450F3B93
:1038E7000F300F250F1A0F0E0F020EF50EE80EDB25
:1038F7000ECC0EBE0EAE0E9F0E8E0E7D0E6C0E5AA9
:103907000E470E340E200E0C0DF70DE20DCB0DB544
:103917000D9D0D850D6D0D540D3A0D200D050CE90E
:103927000CCE0CB10C940C760C580C3A0C1B0BFB00
:103937000BDB0BBB0B9A0B790B570B350B130AF1F0
:103947000ACE0AAB0A870A640A400A1C09F809D496
:1039570009B0098C09670943091F08FB08D608B293
:10396700088E086A0846082307FF07DC07B9079689
:1039770007730751072F070D06EC06CA06AA068923
:1039870006690649062A060A05EC05CD05B0059223
:1039970005750558053C0520050504EA04CF04B55F
:1039A700049C04820469045104390422040B03F4BF
:1039B70003DE03C803B2039D038903750361034D47
:1039C700033B03280316030402F202E102D102C0FB
:1039D70002B002A0029102820273026502570249F5
:1039E700023C022F02220216020901FD01F201E642
:1039F70001DB01D001C601BB01B101A7019D019403
:103A0700018B018201790170016801600158015041
:103A17000148014101390132012B0125011E01181D
:103A27000111010B010500FF00FA0ECF0EBB0EA717
:103A37000E920E7C0E650E4D0E340E190DFE0DE125
:103A47000DC40DA50D850D640D420D1E0CFA0CD489
:103A57000CAE0C860C5D0C330C080BDC0BB00B8228
:103A67000B540B250AF50AC40A930A610A2F09FDAC
:103A770009CA09960963092F08FC08C8089508614F
:103A8700082E07FB07C8079607640733070206D205
:103A970006A206730645061705EA05BF05930569DD
:103AA7000540051704F004C904A3047E045A04372B
:103AB700041503F403D303B403960378035B033FAE
:103AC7000324030A02F002D702BF02A80292027C73
:103AD70002670253023F022C021A020801F701E6AD
:103AE70001D601C701B801A9019C018E01810174AA
:103AF7000168015D01510146013C01320128011FA6
:103B07000115010D010400FC00F400EC00E500DEE6
:103B170000D700D000CA00C300BD00B800B200AD96
:103B270000A700A2009E009900940090008C0087D7
:103B370000840080007C007800750072006E006BC6
:103B47000068006500620060005D005A005800557B
:103B570000530051004E004C004A00480046004404
:103B670000430041003F003E003C003A0039003767
:103B770000360035003300320031002F002E002DB3
:103B8700002C002B002A00290028002700260025EA
:103B97000024002300010C01010402011E030A9600
:103BA700040132050202060064070101080000094A
:103BB700015A0A01040B00030E01010F0001120054
:103BC7006413010114013C1501FA1664FA17FFFF8B
:103BD7001D00072000072400022632962701012C2A
:103BE700000130010132010333000235FFFF3603C4
:103BF700073CFFFF3DFFFF180002191E461A00028F
:103C07001B00022D32C82E00012F013CFAFAFA18C8
:103C1700000019FFFF1A00001B00002D32C82E00FC
:103C2700012F013CFAFAFA18000019FFFF1A0000E9
:0F3C37001B00002DFFFF2EFFFF2FFFFFFAFAFAF1
:10004800E50C901F7DF8282873803475E700A20D11
:10005800B34008E5B54408F5B58006E5B554F7F5AD
:10006800B575E710801975E700A20DB34008E5B52E
:0F0078004402F5B58006E5B554FDF5B575E71002
:091F7D0002005102005302006E43
:100087002290083BE0900041F090083CE090004847
:10009700F090083DE0900049F090083EE090004C59
:1000A700F090083FE090004DF0900840E09000503D
:1000B700F0900841E0900051F0900842E090005C19
:1000C700F0900843E090005EF0900844E0900062F2
:1000D700F0900845E0900064F0900846E0900065D5
:1000E700F0900847E0900066F0900848E0900067BD
:1000F700F0900849E090006AF090084AE090006BA1
:10010700F090084BE090006EF090084CE090007A79
:10011700F090084DE090007BF090084EE090007C56
:10012700F090084FE090007DF0900850E090007E3E
:10013700F0900851E090007FF0900852E090008026
:10014700F0900853E0900081F0900854E09000830D
:10015700F0900855E0900084F0900856E0900085F4
:10016700F0900857E0900086F090007AE090002B1E
:10017700F090007BE090002CF090007CE090002D48
:10018700F090007DE090002EF090007EE090002F30
:10019700F090007FE0900030F0900080E090003118
:1001A700F0900081E0900032F0900083E09000270B
:1001B700F0900084E0900028F0900085E0900029FE
:1001C700F0900086E090002AF0744C90010FF074D4
:1001D70065900110F07478900111F0747590011218
:1001E700F07473900113F07420900114F07441902F
:1001F7000115F07433900116F07434900117F07400
:1002070033900118F07420900119F0743490011A9A
:10021700F0745390011BF0745090011CF0744490DB
:10022700011DF09003BEE09003FEF022900838E035
:10023700FEA3E0FF7463BE0010D39F400C903B9B6E
:1002470012001EE493F599804C90000BE0D39404C0
:100257004014900838E0FEA3E0FF903B9B12001E7D
:10026700E493F599802F90000BE0D394034014900A
:100277000838E0FEA3E0FF903BB312001EE493F5BD
:10028700998012900838E0FEA3E0FF903BCB120064
:100297001EE493F59990083812000E900838E0FE96
:1002A700A3E0FF747B6F4E70037564002290005CBF
:1002B700E0B40105756D028003756D01A206B340B8
:1002C70016900124E0700C900125E070069001263D
:1002D700E060028002C206900124E0B4300F900172
:1002E70025E0B44708900126E0643B60028004D211
:1002F700078002C207E548B4010280030203CE90DB
:10030700007AE090002BF090007BE090002CF090BA
:10031700007CE090002DF090007DE090002EF090A2
:10032700007EE090002FF090007FE0900030F0908A
:100337000080E0900031F0900081E0900032F09072
:100347000083E0900027F0900084E0900028F09070
:100357000085E0900029F0900086E090002AF09058
:100367000063E0B40117900000740FF0A374FFF06E
:10037700900002E4F0A3F07402900063F090006331
:10038700E0B40341900002E0FEA3E0FF900000E02C
:10039700FCA3E0FD1200037410123E167408123E0F
:1003A70008EF900062F0EF700674FF900062F0743F
:1003B70000900063F0900001E0900048F09000008A
:1003C700E0900049F0800990006BE07003754801E8
:1003D7007E887F4D900041E08E048F05FF123DF827
:1003E7008C328D3390004DE075F0FAA4FFAEF0909B
:1003F700004CE08E048F05FF123DF88C368D379048
:100407000039E0F54E900037E0FE900053E0B50666
:1004170018900036E0FE900052E0B5060C900035CB
:10042700E0FE900043E06E606F900053E07006902E
:100437000052E060067400900043F0900053E0B46F
:1004470002089000337401F08005900033E4F090C7
:100457000052E0B402089000347401F08005900067
:1004670034E4F0900052E06006900034E0600280CF
:1004770005754E038003754E04E549B54802D20859
:10048700900052E0900036F0900053E0900037F073
:10049700900043E0900035F07401900088F07400FC
:1004A700900089F0740090008AF0740090008BF03F
:1004B700740090008CF0740090008DF07400900030
:1004C7008EF0740190008FF07400900090F074002B
:1004D700900091F07400900092F07400900093F0F7
:1004E7007400900094F07400900095F074019000EF
:1004F70096F07400900097F07400900098F07400E4
:10050700900099F0740090009AF0740090009BF0AE
:10051700740090009CF0740190034CF074009003F9
:100527004DF0740090034EF0740090034FF0740088
:10053700900350F07400900351F07400900352F050
:10054700740190038CF0740190038DF07400900394
:100557008EF0740090038FF07400900390F0740095
:10056700900391F07400900392F074009003CCF024
:1005770074019003CDF074009003CEF074009003E3
:10058700CFF074009003D0F074009003D1F07400A2
:100597009003D2F0740090040CF0740090040DF0F6
:1005A700740090040EF0740090040FF0740090042F
:1005B70010F07400900411F07400900412F0121FF0
:1005C700A722C2A2C2A1C292C203E5B554FBF5B5E8
:1005D700754304E54304F544900039E0F54E900077
:1005E70026E4F0C205E5B554FEF5B5900026E4F023
:1005F700755000C28E758D00758B0075400075258E
:1006070000752400D28EC296C295C287C2A0C29737
:10061700E5B554BFF5B5E5B554DFF5B5E5B554EF28
:10062700F5B5E5B5547FF5B5E5B554F7F5B5E5B5D9
:1006370054FDF5B522755600755500AE55AF567485
:1006470062BE00039F50030206F9903B9B12001EF7
:10065700E493900038123E2E0FBF00010EE0FC908D
:100667003B9B12001EECFEE493FFEEC39F5026AEA9
:1006770055AF560FBF00010E903B9B12001EAE55A3
:10068700AF56E493FC903B9B12001EE49390003816
:10069700123E2EECF0AE55AF56903B9B12001EE477
:1006A70093900038123E2EE0FC903B9D12001EEC0A
:1006B700FCE493FDECD39D4019903B9D12001EE492
:1006C70093FC903B9B12001EE493900038123E2E41
:1006D700ECF0AE55AF5674022FFF50010E8E558FBA
:1006E700567856740126F6500418E436F64003028D
:1006F700064222755600755500AE55AF567417BEA3
:1007070000039F50030207C7903BFE12001EE493AD
:10071700900038123E2E0FBF00010EE0FC903BFE0A
:1007270012001EECFEE493FFEEC39F5026AE55AFBA
:10073700560FBF00010E903BFE12001EAE55AF567E
:10074700E493FC903BFE12001EE493900038123EA7
:100757002EECF0AE55AF56903BFE12001EE4939080
:100767000038123E2EE0FC903C0012001EECFCE428
:1007770093FDECD39D4019903C0012001EE493FCBE
:10078700903BFE12001EE493900038123E2EECF0D0
:10079700AE55AF5674126F4E7006755618755500E4
:1007A700AE55AF5674022FFF50010E8E558F5678F7
:1007B70056740126F6500418E436F6400302070083
:1007C70022755600755500AE55AF567417BE000317
:1007D7009F5003020895903C1612001EE493900068
:1007E70038123E2E0FBF00010EE0FC903C1612009F
:1007F7001EECFEE493FFEEC39F5026AE55AF560F97
:10080700BF00010E903C1612001EAE55AF56E49382
:10081700FC903C1612001EE493900038123E2EEC1A
:10082700F0AE55AF56903C1612001EE49390003878
:10083700123E2EE0FC903C1812001EECFCE493FDE7
:10084700ECD39D4019903C1812001EE493FC903C99
:100857001612001EE493900038123E2EECF0AE55AF
:10086700AF5674126F4E7006755618755500AE5513
:10087700AF5674022FFF50010E8E558F567856745F
:100887000126F6500418E436F640030207CE227517
:100897005600755500AE55AF567417BE00039F50EE
:1008A70003020963903C2E12001EE4939000381255
:1008B7003E2E0FBF00010EE0FC903C2E12001EECF6
:1008C700FEE493FFEEC39F5026AE55AF560FBF0011
:1008D700010E903C2E12001EAE55AF56E493FC90CD
:1008E7003C2E12001EE493900038123E2EECF0AE20
:1008F70055AF56903C2E12001EE493900038123EDE
:100907002EE0FC903C3012001EECFCE493FDECD38F
:100917009D4019903C3012001EE493FC903C2E122F
:10092700001EE493900038123E2EECF0AE55AF5601
:1009370074126F4E7006755618755500AE55AF5642
:1009470074022FFF50010E8E558F5678567401266C
:10095700F6500418E436F6400302089C2212063CBF
:1009670090F802E493B404051207C8801290F802C5
:10097700E493D3940440051206FA800312089622E2
:100987000541220540220542C2CF2290F800E49398
:100997006406600280FE75840175A70075FF80906C
:1009A700083AE4F075C91075A70F75A1C775A700B8
:1009B70075D90075CEFF75A70F75F1FE75F2FF7536
:1009C700F33775F47875A4BA75A5FF75A60775AEE4
:1009D7000075AFFF75D48175D5FF75D6FF75D7FF45
:1009E700C296C295C2A0C297E5B554BFF5B5E5B5A5
:1009F70054DFF5B5E5B554EFF5B5E5B5547FF5B575
:100A0700E5B554F7F5B5E5B554FDF5B575A700752A
:100A1700A20175A14775F80975BC0175BE0475BDBE
:100A27006C75BE0775BDA075BE0875BD0175BC00A8
:100A370075BB1875BC2075BA0875E88075D1137534
:100A4700A70F75E10575E20075C7407597007597A3
:100A570080740A123DE87597C0E5975420700280AC
:100A6700F8758F0275A700D2AF75980075A90C7538
:100A7700A70F75AB4375ADFB75AC1E75A7007589E0
:100A870011758E00758C00758A00D2A9D28C758D70
:100A970000758B00D2ABD28E75CD0075CC0075CAB0
:100AA7000075CB00D2ADC2CFD2CA75910475920042
:100AB7007593CD75EF0675D94075CF01900838E469
:100AC700F0A3F0756400756500C299D206C20912D9
:100AD70005C97509C87508001220DD75A70FE5FC63
:100AE700900015F0E5FB900016F0E5FA900017F07E
:100AF700E5F9900018F075A70090F800E493F55415
:100B07001221FC12273690F807E493900022F09008
:100B17000022E04408900022F0900022E054FE906A
:100B27000022F0120088900858E0900124F0900805
:100B370059E0900125F090085AE0900126F09001C5
:100B470024E0700C900125E07006900126E0600219
:100B57008004C2068002D2067548017549017403F4
:100B6700900036F01209647400900063F0740090EE
:100B7700006CF01202B47406900008F07400900044
:100B870009F0740290000AF090F802E49390000BC9
:100B9700F090F803E49390000CF090F804E493903D
:100BA700000DF0740590000EF090000BE0B4040601
:100BB700740490000EF090000BE0B40306740390E9
:100BC700000EF0740190000FF07403900010F074A1
:100BD70006900011F07402900012F090F805E4936B
:100BE700900013F090F806E493900014F0740090CE
:100BF7000019F0740090001AF0740090001BF07454
:100C07000090001CF0740090001DF0740090001E0E
:100C1700F0740090001FF07400900020F0740090B2
:100C27000021F074FF900023F0A2B6B39200A2B3A4
:100C3700B39201756A00743A900738F074FD900713
:100C470039F0C208900024E4F0754A007523007556
:100C57002200753D00752900752800753E00754511
:100C6700007546007544017552007551007553CDE6
:100C7700754700753A00753B00753C00753900757E
:100C87003800754D0090000474FDF0A374E8F090EF
:100C97000024E4F07464900025F0754100C294C20A
:100CA70093C287C290C2911220B0C203D2B0D2B70A
:100CB700D2A7D2A6D2B1D2A37E017F00900049E08D
:100CC700123E16900048E02FFF50010E900000EEF4
:100CD700F0A3EFF0EFD394FFEE940F4007900000DE
:100CE700E4F0A3F0900062E0700674FF900062F0F9
:100CF700D29CD2EC75CF01A298B34005C298122AB4
:100D0700E2E5646006A299B3B340028005C2991276
:100D17002EF8E56564016005E565B4040280D5E554
:100D270041D39405400CE54AC394C85002054A755F
:100D37004100E553C394F0501A785112003FAE5169
:100D4700AF52EFD394E8EE94034008055375520071
:100D5700755100C28E7E047F00E540123E16E58D78
:100D670075F004A4FDACF0EF2DFDEE3CFCE58B75B2
:100D7700F04084FF7E00ED2FFFEC3EFE8E248F2592
:100D8700D28EA2B6300001B35003020EE3A2B630F2
:100D97000001B35003020EE3A2B640730545A20952
:100DA700400575FFA0D209E5B54401F5B5900025CA
:100DB700E4F0900041E0C395455052E52545246095
:100DC7000F7C887D4DAE24AF25123C468E228F23A3
:100DD700AE22AF23E53D2FFF50010E7401123E08EE
:100DE7008E228F2385233D754501C28E758D007533
:100DF7008B00754000D28E7403BE00039F5006908F
:100E070000267401F0E56AB40D03756A00D200A2EA
:100E1700B6B35003020EE3900025E4F0C200900041
:100E270055E060077401F508123039900058E0600A
:100E3700077402F508123039E547B40708E5B544E9
:100E470080F5B58006E5B5547FF5B5A203B3400438
:100E5700D2878002C287900043E06004D29080026C
:100E6700C290900034E0B40104D2948002C29490FE
:100E77000033E0B40104D2938002C293A205B340C9
:100E870004D2918002C29190000EE0FE90000BE028
:100E9700C39E400990000BE0D39408400974FB906F
:100EA7000024F01205C990000CE0601590000CE0DA
:100EB700FE90000AE06E600974FC900024F01205B1
:100EC700C990000DE0601590000DE0FE90000FE066
:100ED7006E600974FE900024F01205C9C2CA7E0133
:100EE7007F00E542123E16E5CD2FFF50010E8E26FC
:100EF7008F27D2CA900066E0B40148900004E0FC56
:100F0700A3E0FDEFC39DEE9C4039B204E5294528D7
:100F17006013A204B34008E5B54404F5B58006E5BF
:100F2700B554FBF5B5900004E0FEA3E0FF90000682
:100F3700E0FCA3E0FDEF2DFDEE3CFC900004ECF09F
:100F4700A3EDF0A2B3300101B35003021043A2B3E3
:100F5700300101B35003021043A2B3500302103C07
:100F67000546A209400575FFA0D209E5B54401F57C
:100F7700B5900025E4F090004CE0C395464003028D
:100F8700103AE5274526600F7CEA7D60AE26AF273D
:100F9700123C468E288F29AE28AF2990004DE012CB
:100FA7003E1674FF8E048F05FF123DF88C288D299D
:100FB700E53E2DFD50010C74018C068D07123E088D
:100FC7008E288F2985293EA205B340157464123EE9
:100FD70016900051E08E048F05FF123DF88C288D86
:100FE70029754601900004E0FEA3E0FFAC26AD277B
:100FF700120003900004EEF0A3EFF0900067E0FF0B
:10100700123DF8740AFF123DF8900065E08C068DDA
:1010170007123E1674148E048F05FF123DF89000D8
:1010270006ECF0A3EDF0C2CA75CD0075CC00754291
:1010370000D2CAD201A2B3B34002C201900026E097
:10104700B40107E547C394064003021657E55090DD
:101057001F86F8282873900043E0C39402400302D8
:1010670011B1E543D3940150030211B1E54375F083
:1010770040A4FFAEF09002FC12001EE0C3953B5067
:1010870018E54375F040A4FFAEF09002FB12001E76
:10109700E0F52D752C000211B1E54375F040A4FF72
:1010A700AEF09002FA12001EE0C3953B4003021116
:1010B7004DE54375F040A4FFAEF09002FB12001E11
:1010C700E54375F040A4FFAEF0E0FC9002F9120092
:1010D7001EECFEE0FFEEC39FFEE5438E0475F04075
:1010E700A4FFAEF09002FA12001EE0F404253B8C38
:1010F7000088F0A4FFAEF0E5438F048E0575F0403D
:10110700A4FFAEF09002FC12001EE54375F040A468
:10111700FFAEF0E0FA9002FA12001EEAFEE0FFEEE0
:10112700C39FFECDCCCD8E07123DF8E54375F04049
:10113700A4FFAEF09002F912001EE02DFD50010C45
:101147008C2C8D2D8064E54375F040A4FFAEF090A4
:1011570002F912001EE54375F040A4FFAEF0E0FC73
:101167009002F812001EECFEE0FFEEC39F853BF0F5
:10117700A4FFAEF0E5438F048E0575F040A4FFAEE3
:10118700F09002FA12001EE0FECDCCCD8E07123D84
:10119700F8E54375F040A4FFAEF09002F812001E88
:1011A700E02DFD50010C8C2C8D2D7550010216572A
:1011B700900043E0C394024003021365900039E0B6
:1011C700D39543500302130DE54375F040A4FFAEDA
:1011D700F090030212001EE0C3953B5018E54375DB
:1011E700F040A4FFAEF090030112001EE0F52B754E
:1011F7002A0002130DE54375F040A4FFAEF09003FB
:101207000012001EE0C3953B40030212A9E5437597
:10121700F040A4FFAEF090030112001EE54375F005
:1012270040A4FFAEF0E0FC9002FF12001EECFEE0CF
:10123700FFEEC39FFEE5438E0475F040A4FFAEF0BA
:1012470090030012001EE0F404253B8C0088F0A4F4
:10125700FFAEF0E5438F048E0575F040A4FFAEF0B6
:1012670090030212001EE54375F040A4FFAEF0E0C4
:10127700FA90030012001EEAFEE0FFEEC39FFECDC8
:10128700CCCD8E07123DF8E54375F040A4FFAEF0D4
:101297009002FF12001EE02DFD50010C8C2A8D2BB1
:1012A7008064E54375F040A4FFAEF09002FF1200A2
:1012B7001EE54375F040A4FFAEF0E0FC9002FE127D
:1012C700001EECFEE0FFEEC39F853BF0A4FFAEF0EF
:1012D700E5438F048E0575F040A4FFAEF090030040
:1012E70012001EE0FECDCCCD8E07123DF8E543750A
:1012F700F040A4FFAEF09002FE12001EE02DFD505C
:10130700010C8C2A8D2BE543B40123E54ED39401C0
:10131700401CE54704D395434014E53BC39405506F
:101327000D900349E0A828B80006952940028003DC
:10133700754302E543B54E22900039E0D39543400B
:1013470019E54375F040A4FFAEF090030112001EAB
:10135700E0A822B80006952340028002054E75508A
:1013670002021657900043E0B4022AE54375F040A5
:10137700A4FFAEF090030112001EE0F52B752A00C2
:10138700E54375F040A4FFAEF09002F812001EE0AE
:10139700F52D752C00900043E0B4030F90003BE05F
:1013A700F52B752A00752D00752C00755003021654
:1013B70057E54375F040A4FFAEF090030A12001EF4
:1013C700E0C3954A400302148D900033E07036E580
:1013D70043D394014029AE22AF23AC2CAD2DEDD3DE
:1013E7009FEC9E401AE54375F040A4FFAEF09003D2
:1013F7000812001EE0A828B80005D39529500280DE
:101407000215438034E543D394024029AE22AF232B
:10141700AC2CAD2DEDD39FEC9E401AE54375F04003
:10142700A4FFAEF090030812001EE0A828B800053C
:10143700D39529500280021543E543B54437E54368
:10144700C3954E5030E54704D395434028AE22AFAD
:1014570023AC2AAD2BEFD39DEE9C4019E54375F0E5
:1014670040A4FFAEF090030912001EE0A828B800C0
:10147700069529400280020543C292E54365446010
:1014870005C203754A00755004021657E54375F007
:1014970040A4FFAEF090030412001EE0B40117E56C
:1014A7004375F040A4FFAEF090030A12001EE0243B
:1014B7000AC3954A4003021563752F64752E00A26F
:1014C70003B3500B90004AE02405C3953B40030249
:1014D7001563E54375F040A4FFAEF09003071200D3
:1014E7001EE0C3953B4064E54375F040A4FFAEF0B2
:1014F70090030612001EE54375F040A4FFAEF0E02E
:10150700FC90030512001EECFEE0FFEEC39F853B37
:10151700F0A4FFAEF0E5438F048E0575F040A4FFFD
:10152700AEF090030712001EE0FECDCCCD8E071261
:101537003DF8E54375F040A4FFAEF09003051200B7
:101547001EE02DFD50010C8C2E8D2FAE22AF23AC4B
:101557002EAD2FEFD39DEE9C4002D20375500502AE
:101567001657E543B40109900043E0C394024003D2
:10157700021637900342E0D3953B5003021637908B
:101587000340E0C3953B5040900341E0FE90033F8A
:10159700E0F4042EFE900340E0F404253B8E00881F
:1015A700F0A4FFAEF0900342E0FC900340E0F404A7
:1015B7002C8E048F05FF123DF890033FE02DFD5060
:1015C700010C8C2A8D2B802C90033FE0FE90033E6C
:1015D700E0F4042E853BF0A4FFAEF0900340E08ECC
:1015E700048F05FF123DF890033EE02DFD50010CDE
:1015F7008C2A8D2BE543C3954E5030E54704D39590
:10160700434028AE22AF23AC2AAD2BEFD39DEE9CEF
:101617004019E54375F040A4FFAEF09003091200AE
:101627001EE0A828B80006952940028003754302EA
:10163700900033E0B40106E543640160028003755E
:101647004302E54365446005C203754A00755000CF
:101F860002105D0211B702136B0213B8021493021A
:021F96001569CB
:1016570090003AE02402A822B80007D3952340025D
:10166700C203900026E0B40109900043E0C394034D
:1016770040030217DF900033E0600302172EE543B3
:10168700D394014034E54375F040A4FFAEF09002D7
:10169700FE12001EE0A822B8001FD39523401AE5CA
:1016A7004375F040A4FFAEF090030912001EE0A8B6
:1016B70028B80005D39529500280021543E543D386
:1016C7009401402FE54375F040A4FFAEF09002FC73
:1016D70012001EE0C3953B501AE54375F040A4FF86
:1016E700AEF090030812001EE0A828B80005D395B5
:1016F70029500280021543E543D394014022E54770
:1017070004C39543501AE54375F040A4FFAEF0902B
:10171700030812001EE0A828B80005D39529500237
:10172700800215430217D4E543D394024034E543BE
:1017370075F040A4FFAEF09002FE12001EE0A82252
:10174700B8001FD39523401AE54375F040A4FFAEB8
:10175700F090030912001EE0A828B80005D39529C8
:10176700500280021543E543D39402402FE54375A9
:10177700F040A4FFAEF09002FC12001EE0C3953BC0
:10178700501AE54375F040A4FFAEF090030812002D
:101797001EE0A828B80005D39529500280021543FA
:1017A700E543D394024022E54704C39543501AE525
:1017B7004375F040A4FFAEF090030812001EE0A8A6
:1017C70028B80005D39529500280021543E54365E3
:1017D700446005C203754A0090004AE0D3953B5028
:1017E7000990003EE0C3953B5002C203900043E0DE
:1017F7007003021A46A2A5B34008A2A4B34003028D
:101807001A2FAE30AF317441D39F749C9E40057838
:101817003012003FAE30AF31EFB48806EEB413029A
:101827008003021A0AA2A550030218CD900043E0D4
:10183700B4010B900039E0D3954E4002054E90005D
:1018470043E0B40254E54375F040A4FFAEF09003C3
:101857000A12001EE0C3954A503F900039E0D39525
:10186700434021E54704D395434019E54375F040CC
:10187700A4FFAEF09002FE12001EE0A822B80006F8
:101887009523400280020543900039E0F54EE54379
:1018970065446005C203754A00900043E0B403261F
:1018A700900039E0D395434008E54704D39543506A
:1018B7000280020543900039E0F54EE54365446038
:1018C70005C203754A00A2A45003021A0A900043F6
:1018D700E0B4016E900033E07035E543D3940140E6
:1018E70029E54375F040A4FFAEF090030812001EEF
:1018F700E0A828B8000FD39529400A1543754A0078
:1019070085434E800385434E8003754E018033E542
:1019170043D394024029E54375F040A4FFAEF0900D
:10192700030812001EE0A828B8000FD39529400A23
:101937001543754A0085434E800385434E800375E2
:101947004E02900043E0D3940150030219FEE54391
:1019570075F040A4FFAEF090030A12001EE0C39595
:101967004A40030219FE900033E07041E543D394E7
:10197700014034E54375F040A4FFAEF09002FB123E
:10198700001EE0A822B8001FD39523401AE543752F
:10199700F040A4FFAEF090030812001EE0A828B89C
:1019A7000005D39529500280021543803FE543D3B4
:1019B70094024034E54375F040A4FFAEF09002FB7B
:1019C70012001EE0A822B8001FD39523401AE54352
:1019D70075F040A4FFAEF090030812001EE0A8289F
:1019E700B80005D39529500280021543E5436544A5
:1019F7006005C203754A00E547B40704054D800337
:101A0700754D0090006BE0B4010EAE30AF31EF645E
:101A1700407005EE649C6002800EA2A540037548E5
:101A270001A2A44003754802A2A5B3B35006A2A41D
:101A3700B3B340028006753100753000021B34A233
:101A4700A5B34008A2A4B34003021B20AE30AF31B8
:101A57007441D39F749C9E4005783012003FAE308E
:101A6700AF31EFB48806EEB413028003021B20A245
:101A7700A5406F900052E0605A900034E0B401072F
:101A8700900034E4F080069000347401F090003444
:101A9700E07005754E038003754E04900034E0B482
:101AA7000104D2948002C294E543B4041AE5437555
:101AB700F040A4FFAEF090030812001EE0A828B87B
:101AC7000005D3952950028008754303C203754A60
:101AD700008003754E04E547B40704054D80037580
:101AE7004D00A2A44033900053E06021900033E002
:101AF700B40107900033E4F080069000337401F0DE
:101B0700900033E0B40104D2938002C293E547B456
:101B17000704054D8003754D00A2A5B3B35006A277
:101B2700A4B3B340028006753100753000E54865FF
:101B370049600690006CE06002802CE548901F9891
:101B4700F82828738012122736800D122821800862
:081B570012290C80031229F78A
:0F1F9800021B4B021B4D021B52021B57021B5C0C
:101B5F001200881202B4854849741B900024F0E5E6
:101B6F0047C394065005E543B54402804EC203E5D2
:101B7F004375F040A4FFAEF090030C12001EE0304E
:101B8F00E003D38001C39296E54375F040A4FFAE06
:101B9F00F090030D12001EE030E003D38001C392DA
:101BAF0095854344AE28AF297405BE00039F5007A7
:101BBF00E53BD3940550028002D292E547D39405BA
:101BCF005003021C93C203E543D394014059E543EC
:101BDF0075F040A4FFAEF090030812001EE0A82895
:101BEF00B80007D3952940021543E5436544603596
:101BFF00E54375F040A4FFAEF090030C12001EE019
:101C0F0030E003D38001C39296E54375F040A4FF03
:101C1F00AEF090030D12001EE030E003D38001C33D
:101C2F009295854344805DE547B4061A900096E08F
:101C3F0030E003D38001C39296900097E030E00329
:101C4F00D38001C39295E547B4071A90008FE03017
:101C5F00E003D38001C39296900090E030E003D36D
:101C6F008001C39295E547B4081A900088E030E0F0
:101C7F0003D38001C39296900089E030E003D380B4
:101C8F0001C39295E54764066005E547B40808E58A
:101C9F00B54410F5B58006E5B554EFF5B590005C89
:101CAF00E06058E53B75F00284FF7E00900138122A
:101CBF00001EE0F54BE53C75F00A84FF7E009002B4
:101CCF003812001EE0F54CE54B254CD39464400BC5
:101CDF00E54B254CC39464F54B8003754B00E54BE6
:101CEF0075F00284FF7E008F4BEFC394335007EFE4
:101CFF0024CDF54B8003754BFF801CE53B75F0023F
:101D0F0084FF7E0090013812001EE075F00284FF00
:101D1F007E00EF24CDF54BE595C3954B4004C2A251
:101D2F008002D2A2A203B34005E547B4070375535F
:101D3F00CDE595C395534004C2A18002D2A1E56AB7
:101D4F00C3940D501DE56A75F00284AFF07E00EF6D
:101D5F004E700512327F800AA2EDB34005C2ED121C
:101D6F00327FE54DD394045003021E5975CF01C243
:101D7F00A2AE30AF317488D39F74139E4005A2A5D5
:101D8F00B34014AE30AF317488D39F74139E4005A7
:101D9F00A2A4B340028048783012003FAE30AF317A
:101DAF00EFB4883BEEB41337A2A5B35009900039B6
:101DBF00E0D395435002800405438011A2A5B35090
:101DCF0008900039E0654360028002D203A2A4B3F9
:101DDF005007E543D39401500280041543C203A278
:101DEF00A5B3B35006A2A4B3B34002800675310069
:101DFF00753000E54365446035E54375F040A4FF59
:101E0F00AEF090030C12001EE030E003D38001C34C
:101E1F009296E54375F040A4FFAEF090030D1200CB
:101E2F001EE030E003D38001C39295854344A203A3
:101E3F0040057553CD80037553FFE595C39553400A
:101E4F0004C2A18002D2A1021D7BA209B3500DAE24
:101E5F0024AF2574E8C39F74039E4002800575FF6D
:101E6F00A0D209AE24AF25EFD39420EE944E5003A9
:101E7F00021F511205C9C28E758D00758B007540FA
:101E8F0000D28EC2037552007551007553CD754344
:101E9F0004752300752200754500754A00C28790AE
:101EAF000043E06004D2908002C290900034E0B40E
:101EBF000104D2948002C294900033E0B40104D2A2
:101ECF00938002C293A205B34004D2918002C291C3
:101EDF00900055E060077401F508123039900058F2
:101EEF00E060077402F508123039E547B40708E5DA
:101EFF00B54480F5B58006E5B5547FF5B59000047F
:101F0F0074FDF0A374E8F0E56AB40D03756A00750B
:101F1F002500752400758D00758B007540009000AD
:101F2F0025E0C394035008900025E004F080067468
:101F3F0003900025F0900025E0B40306E5B554FEAC
:101F4F00F5B5AE26AF27EFD39410EE9427401CC201
:101F5F00CA75CD0075CC00752700752600D2CA75DD
:0E1F6F004200752900752800754600020CFB23
:103D270000000100013201640196019602000212AF
:103D370002240200020003000340038003C00400C2
:103D47000440048004C005000600060006000600C3
:103D5700060006000600060000FF01310163019519
:103D670001FF01FF0211022302FF02FF02FF033FCF
:103D7700037F03BF03FF043F047F04BF04FF05FF66
:103D870006FF06FF06FF06FF06FF06FF06FF06FF04
:101FA700900041E090083BF0900048E090083CF03A
:101FB700900049E090083DF090004CE090083EF01A
:101FC70090004DE090083FF0900050E0900840F0FE
:101FD700900051E0900841F090005CE0900842F0DA
:101FE70090005EE0900843F0900062E0900844F0B3
:101FF700900064E0900845F0900065E0900846F096
:10200700900066E0900847F0900067E0900848F07D
:1020170090006AE0900849F090006BE090084AF061
:1020270090006DE090084BF090006EE090084CF047
:1020370090007AE090084DF090007BE090084EF019
:1020470090007CE090084FF090007DE0900850F001
:1020570090007EE0900851F090007FE0900852F0E9
:10206700900080E0900853F0900081E0900854F0D1
:10207700900083E0900855F0900084E0900856F0B7
:10208700900085E0900857F0900086E0900858F09F
:10209700900124E0900859F0900125E090085AF04B
:1020A700900126E090085BF022900838E4F0A3F056
:1020B700755A00755900756400756500C20AD20B20
:1020C700755E00755D0075603C755F00756B00752A
:1020D7006C0075690022750B00750A00AE0AAF0B1C
:1020E700AC08AD09EDC39FEC9E401674FF123DE8A6
:1020F70075CF01780B740126F6500418E436F650B4
:10210700DB22C2AF75D900758F0375B7A575B7F117
:1021170090F800E4F0758F0175B7A575B7F1E55430
:1021270090F800F075B7A575B7F190F801E4F07570
:10213700B7A575B7F1900877E090F802F075B7A5E5
:1021470075B7F190087BE090F803F075B7A575B700
:10215700F1900878E090F804F075B7A575B7F1909D
:102167000879E090F805F075B7A575B7F190087A8A
:10217700E090F806F075B7A575B7F190087CE09088
:10218700F807F0758F0075D940D2AF2290083AE072
:10219700B4AB61C2AF75D90075B62275F522758FDC
:1021A7000375B7A575B7F1740090F600F0758F0148
:1021B700755600755500AE55AF56743BBE00279F48
:1021C700402475B7A575B7F190083B12001EE0FCD7
:1021D70090F60012001EECF07856740126F65004B3
:1021E70018E436F650D0758F0075F51175B6207561
:1021F700D940D2AF22C2AF75D90075F52275560006
:10220700755500AE55AF56743BBE00229F401F90D8
:10221700F60012001EE493FC90083B12001EECF03F
:102227007856740126F6500418E436F650D575F53D
:102237001175D940D2AF2290083AE0B4AA028003C0
:1022470002237BC2AF75D90075B62275F522758F4B
:102257000375B7A575B7F1740090EE00F075B7A5D3
:1022670075B7F1740090F000F075B7A575B7F17404
:102277000090F200F075B7A575B7F1740090F400FF
:10228700F0758F01755600755500AE55AF5674FF42
:10229700C39F74019E402475B7A575B7F1900038A8
:1022A70012001EE0FC90EE0012001EECF07856744F
:1022B7000126F6500418E436F650CF7556007555CA
:1022C70000AE55AF5674FFC39F74019E402475B787
:1022D700A575B7F190023812001EE0FC90F00012CD
:1022E700001EECF07856740126F6500418E436F612
:1022F70050CF755600755500AE55AF5674FFC39F46
:1023070074019E402475B7A575B7F1900438120083
:102317001EE0FC90F20012001EECF07856740126C5
:10232700F6500418E436F650CF755600755500AED2
:1023370055AF5674FFC39F74019E402475B7A575AA
:10234700B7F190063812001EE0FC90F40012001E50
:10235700ECF07856740126F6500418E436F650CFA0
:10236700758F0075F51175B62075D940D2AF743ADF
:10237700900738F02290083AE0B4AA0280030224BA
:10238700B9C2AF75D90075B62275F522758F037579
:10239700B7A575B7F1740090E600F075B7A575B7E6
:1023A700F1740090E800F075B7A575B7F174009067
:1023B700EA00F075B7A575B7F1740090EC00F075F9
:1023C7008F01755600755500AE55AF5674FFC39F04
:1023D70074019E402475B7A575B7F19000381200B7
:1023E7001EE0FC90E60012001EECF0785674012601
:1023F700F6500418E436F650CF755600755500AE02
:1024070055AF5674FFC39F74019E402475B7A575D9
:10241700B7F190023812001EE0FC90E80012001E8F
:10242700ECF07856740126F6500418E436F650CFCF
:10243700755600755500AE55AF5674FFC39F7401AE
:102447009E402475B7A575B7F190043812001EE0B9
:10245700FC90EA0012001EECF07856740126F65044
:102467000418E436F650CF755600755500AE55AFD3
:102477005674FFC39F74019E402475B7A575B7F1C5
:1024870090063812001EE0FC90EC0012001EECF0E3
:102497007856740126F6500418E436F650CF758F37
:1024A7000075F51175B62075D940D2AF743A90070B
:1024B70038F02290083AE0B4AA0280030225F7C256
:1024C700AF75D90075B62275F522758F0375B7A557
:1024D70075B7F1740090DE00F075B7A575B7F174A4
:1024E7000090E000F075B7A575B7F1740090E200B1
:1024F700F075B7A575B7F1740090E400F0758F011A
:10250700755600755500AE55AF5674FFC39F7401DD
:102517009E402475B7A575B7F190003812001EE0EC
:10252700FC90DE0012001EECF07856740126F6507F
:102537000418E436F650CF755600755500AE55AF02
:102547005674FFC39F74019E402475B7A575B7F1F4
:1025570090023812001EE0FC90E00012001EECF022
:102567007856740126F6500418E436F650CF75569F
:1025770000755500AE55AF5674FFC39F74019E405A
:102587002475B7A575B7F190043812001EE0FC90CA
:10259700E20012001EECF07856740126F65004187B
:1025A700E436F650CF755600755500AE55AF5674E4
:1025B700FFC39F74019E402475B7A575B7F19006B8
:1025C7003812001EE0FC90E40012001EECF0785672
:1025D700740126F6500418E436F650CF758F00754F
:1025E700F51175B62075D940D2AF743A900738F017
:1025F7002290083AE0B4AA028003022735C2AF75D9
:10260700D90075B62275F522758F0375B7A575B70D
:10261700F1740090D600F075B7A575B7F174009006
:10262700D800F075B7A575B7F1740090DA00F075AA
:10263700B7A575B7F1740090DC00F0758F0175567A
:1026470000755500AE55AF5674FFC39F74019E4089
:102657002475B7A575B7F190003812001EE0FC90FD
:10266700D60012001EECF07856740126F6500418B6
:10267700E436F650CF755600755500AE55AF567413
:10268700FFC39F74019E402475B7A575B7F19002EB
:102697003812001EE0FC90D80012001EECF07856AD
:1026A700740126F6500418E436F650CF75560075B7
:1026B7005500AE55AF5674FFC39F74019E402475F5
:1026C700B7A575B7F190043812001EE0FC90DA0048
:1026D70012001EECF07856740126F6500418E43602
:1026E700F650CF755600755500AE55AF5674FFC3FB
:1026F7009F74019E402475B7A575B7F190063812EF
:10270700001EE0FC90DC0012001EECF0785674010D
:1027170026F6500418E436F650CF758F0075F5117C
:1027270075B62075D940D2AF743A900738F022C2F7
:10273700AF75D90075F522755600755500AE55AFC2
:102747005674FFC39F74019E401F90EE0012001E37
:10275700E493FC90003812001EECF07856740126C2
:10276700F6500418E436F650D4755600755500AE89
:1027770055AF5674FFC39F74019E401F90F000121F
:10278700001EE493FC90023812001EECF078567499
:102797000126F6500418E436F650D47556007555E0
:1027A70000AE55AF5674FFC39F74019E401F90F251
:1027B7000012001EE493FC90043812001EECF0781F
:1027C70056740126F6500418E436F650D4755600B0
:1027D700755500AE55AF5674FFC39F74019E401FD9
:1027E70090F40012001EE493FC90063812001EECD1
:1027F700F07856740126F6500418E436F650D4756E
:10280700F51175D940D2AF740090006CF074019047
:102817000042F0743A900738F022C2AF75D90075BC
:10282700F522755600755500AE55AF5674FFC39F18
:1028370074019E401F90E60012001EE493FC900076
:102847003812001EECF07856740126F6500418E48E
:1028570036F650D4755600755500AE55AF5674FF11
:10286700C39F74019E401F90E80012001EE493FC72
:1028770090023812001EECF07856740126F65004C8
:1028870018E436F650D4755600755500AE55AF5658
:1028970074FFC39F74019E401F90EA0012001EE45C
:1028A70093FC90043812001EECF07856740126F65B
:1028B700500418E436F650D4755600755500AE55D9
:1028C700AF5674FFC39F74019E401F90EC00120027
:1028D7001EE493FC90063812001EECF07856740143
:1028E70026F6500418E436F650D475F51175D9401C
:1028F700D2AF740090006CF07402900042F0743A0A
:10290700900738F022C2AF75D90075F522755600C9
:10291700755500AE55AF5674FFC39F74019E401F97
:1029270090DE0012001EE493FC90003812001EECAB
:10293700F07856740126F6500418E436F650D4752C
:102947005600755500AE55AF5674FFC39F74019E70
:10295700401F90E00012001EE493FC900238120022
:102967001EECF07856740126F6500418E436F6503B
:10297700D4755600755500AE55AF5674FFC39F7496
:10298700019E401F90E20012001EE493FC90043861
:1029970012001EECF07856740126F6500418E4363F
:1029A700F650D4755600755500AE55AF5674FFC333
:1029B7009F74019E401F90E40012001EE493FC9058
:1029C700063812001EECF07856740126F6500418EB
:1029D700E436F650D475F51175D940D2AF7400902E
:1029E700006CF07403900042F0743A900738F022BC
:1029F700C2AF75D90075F522755600755500AE55ED
:102A0700AF5674FFC39F74019E401F90D6001200FB
:102A17001EE493FC90003812001EECF07856740107
:102A270026F6500418E436F650D47556007555004E
:102A3700AE55AF5674FFC39F74019E401F90D800D8
:102A470012001EE493FC90023812001EECF0785638
:102A5700740126F6500418E436F650D475560075FE
:102A67005500AE55AF5674FFC39F74019E401F902B
:102A7700DA0012001EE493FC90043812001EECF0FA
:102A87007856740126F6500418E436F650D4755675
:102A970000755500AE55AF5674FFC39F74019E4035
:102AA7001F90DC0012001EE493FC90063812001EF3
:102AB700ECF07856740126F6500418E436F650D434
:102AC70075F51175D940D2AF740090006CF074049D
:102AD700900042F0743A900738F022E5656404608C
:102AE70006E59964FF60028031A20A4004D20A8099
:102AF70027E565600874E62565900024F0E56460C5
:102B07000874F02564900024F0E565B4010280FEA6
:102B1700756500756400C20A8002C20AE5659038CF
:102B27001CF8282873756500E599B4FF03756401DF
:102B3700E599B4FE03756402E599B4FD0375640372
:102B4700E599B4FC03756404E599B4FA0375640563
:102B5700E599B4FB067565011205C9E599B4F9064F
:102B67007565041205C9E599B4F7411205C9C29CF8
:102B770074AB90083AF012219374AA90083AF0E5E2
:012B87004805
:03381C00022B2C50
:102B880090387CF8282873801212223E800D122378
:0B2B98007C80081224BA80031225F88C
:0F387C00022B8F022B91022B96022B9B022BA06B
:102BA30090083AE4F0D29C7565007564007599F756
:102BB300E599D394E54007E599C394F04002801664
:102BC3008599667565027E017F00E566C394E6120A
:102BD3003E168E5B8F5C900838E4F0A3F0E599D342
:102BE30094C44007E599C394E6400280288599661A
:102BF30075650374E5C39566F55C755B00AE5BAF05
:102C03005C903D2712002EE493F8740193900838EA
:102C1300C8F0A3C8F0D299022EF7900838E0FEA3BB
:102C2300E0FF90003812001EE599F090083812007A
:102C33000E900838E0FEA3E0FFEFB40106EEB40700
:102C4300028003022D05900738E0B43C02800302A2
:102C53002D05120964A206B35005A207B3400280F2
:102C630053C29C1200881202B4900124E0900859C8
:102C7300F0900125E090085AF0900126E090085B5F
:102C8300F074AB90083AF012219374AA90083AF0CA
:022C9300E54812
:03381F00022C1D5B
:102C950090388BF8282873801212223E800D12235B
:0B2CA5007C80081224BA80031225F87E
:0F388B00022C9C022C9E022CA3022CA8022CAD16
:102CB00090083AE4F08043C29C121FA77400900869
:102CC00059F0740090085AF0740090085BF074ABEF
:102CD00090083AF012219374AA90083AF012223E1A
:102CE00012237C1224BA1225F8D29C7599FB7464C5
:102CF000F5097508001220DD80FED29C756500750F
:102D000064007599FB022EF7900838E0FEA3E0FFFF
:102D1000EF4E700685995A755900900838E0FEA369
:102D2000E0FF74016F4E701BAC59AD5AAA5BAB5CEF
:102D3000ED2BFBEC3AFA8A068B0790003812001E46
:102D4000E599F090083812000E900838E0FEA3E0F4
:102D5000FF74026F4E700C1202B48566997565009F
:102D6000756400022EF7900838E0FEA3E0FF9000A3
:102D70003812001EE599F090083812000E900838BD
:102D8000E0FEA3E0FFAC5BAD5C8F028E038C068D92
:102D900007903D5F12002EE493F9740193FEEAD38D
:102DA0009EEB994009856699756500756400022E51
:102DB000F7900838E0FEA3E0FF90003812001EE50F
:102DC00099F090083812000E900838E0FEA3E0FF5A
:102DD000EFB40006EEB401028003022EF790001853
:102DE000E0D394C7400B900018E0C394C8F5678007
:102DF0001A900018E0D39463400B900018E0C3943D
:102E000064F5678006900018E0F567E56775F002E5
:102E1000A4FFAEF08F63EF900038123E2EEFFCE07F
:102E2000FDEC90003B123E2EEDFCE0FDEC2DB56775
:102E3000028003022EE80FEF900038123E2EE56369
:102E4000FFE0FCEF90003C123E2EECFFE0FCEFC3F5
:102E50009CB567028003022EE8E56390003A123EBB
:102E60002EE563FFE0FCEF90003D123E2EECFFE00C
:102E7000FCEF2CB56772E56390003E123E2EE0C376
:102E80009567900877F0E56390003F123E2EE0C30F
:102E90009567900878F0E563900042123E2EE0C3FB
:102EA0009567900879F0E563900043123E2EE0C3E9
:102EB000956790087AF0E563900044123E2EE0C3D7
:102EC000956790087BF0E563900045123E2EE0C3C5
:102ED000956790087CF01221097599F97464F509D9
:102EE0007508001220DD80FE7599FF7464F5097580
:072EF00008001220DD80FE46
:09382200022D08022D66022DB1F1
:102EF70022E56490382BF828287302303890083878
:102F0700E0FEA3E0FF90000812001EE0F59990088C
:102F17003812000E900838E0FEA3E0FF741C6F4ED5
:102F27007003756400023038854F99023038900875
:102F370038E0FEA3E0FF90003812001EE0F599EF9D
:102F4700B40107EEB4070375640090083812000E49
:072F5700023038900839E058
:0F382B00022F01022F04022F2F022F35022F5AD6
:102F5E0090389AF828287385239902302D8529995F
:102F6E0002302D853A9902302D853C9902302D85FF
:102F7E00439902302D854E9902302D8547990230A6
:102F8E002D85489902302D756800900053E070062B
:102F9E00900052E060028016A2A44006E568440448
:102FAE00F568A2A54006E5684402F568801A90000F
:102FBE0034E0B40106E5684410F568900033E0B4DF
:102FCE000106E5684420F568A203B34006E56844AF
:102FDE0001F568A205B34006E5684408F568856802
:102FEE0099803CA20BB340077599FAC20B8017A2C9
:102FFE0008B3400575990F800B900024E0F5999069
:10300E000024E4F0C20880178539998012853F9913
:0F301E00800D85699980087599FC8003756400A1
:10389A00022F65022F6B022F71022F77022F7D02F2
:1038AA002F83022F89022F8F022F95022FF10230C8
:0D38BA001602301B02302002302502302A99
:0B302D0090083812000E8003120233DE
:03383A0002303524
:1030380022E50875F003A4FFAEF0EF241AF509E5C0
:103048000904F50AE5092402F50BE5099000381290
:103058003E2EE090383DF828287380218523618032
:103068001C8529618017853A618012853C61800D35
:0D30780085436180088547618003854861BC
:10383D0002306202306402306902306E023073026F
:08384D00307802307D02308268
:10308500E50A900038123E2EE50BFEE0FFEE9000BB
:1030950038123E2EEFFEE0FFEED39F400302319340
:1030A500E509900038123E2EE0D394044051E50A1C
:1030B500900038123E2EE0D39561500EE50B90003E
:1030C50038123E2EE0C395615002800AE508F50CE2
:1030D500D3920D120048E50A900038123E2EE0D337
:1030E5009561500EE50B900038123E2EE0C39561B8
:1030F500500AE508F50CC3920D120048023190E51F
:1031050009900038123E2EE0B40432E50B900038E9
:10311500123E2EE0C39561500AE508F50CD3920DD9
:10312500120048E50A900038123E2EE0D395614022
:103135000AE508F50CC3920D120048804EE50A9089
:103145000038123E2EE0C39561500EE50B90003815
:10315500123E2EE0D395615002800AE508F50CD3A6
:10316500920D120048E50A900038123E2EE0D395E4
:1031750061500EE50B900038123E2EE0C39561506C
:103185000AE508F50CC3920D12004802327EE509E6
:10319500900038123E2EE0D394044051E50A900089
:1031A50038123E2EE0C39561400EE50B90003812B3
:1031B5003E2EE0D395614002800AE508F50CC392E6
:1031C5000D120048E50A900038123E2EE0C39561C5
:1031D500400EE50B900038123E2EE0D39561400A73
:1031E500E508F50CD3920D12004802327EE50990F0
:1031F5000038123E2EE0B40432E50A900038123E43
:103205002EE0C39561500AE508F50CC3920D120036
:1032150048E50B900038123E2EE0D39561400AE553
:1032250008F50CD3920D120048804EE50A9000383F
:10323500123E2EE0C39561400EE50B900038123E1C
:103245002EE0D39561400AE508F50CD3920D1200E6
:1032550048E50A900038123E2EE0D39561400EE510
:103265000B900038123E2EE0C395614002800AE5BE
:1032750008F50CC3920D12004822E56A903855F8FE
:103285002828730238097E017F00E5BE123E16E547
:10329500BD2FFF50010E8E578F58900064E0B4018A
:1032A5000F7E0F7FFFAC57AD581200038E578F5816
:1032B500900063E0B40245AE57AF58900000E0FCC3
:1032C500A3E0FDEDD39FEC9E400A900000E557F08A
:1032D500A3E558F0AE57AF58900002E0FCA3E0FD1F
:1032E500EFD39DEE9C400A900002E557F0A3E55808
:1032F500F0AE57AF587404123E088F3A900063E061
:103305007058AE57AF58900000E0FCA3E0FDEFD336
:103315009DEE9C40091200038E578F588006755804
:1033250000755700900062E0700674FF900062F02F
:10333500AE57AF587410123E16900062E08E048F9F
:1033450005FF123DF88C578D587400D39D74019C70
:10335500400585583A8003753AFFE53A75F00AA4A9
:10336500FFAEF074198E048F05FF123DF88D3BED0D
:10337500255EFFAE5D50010E7401123E088F3B8540
:103385003B5E755D00EFD394624003753B62900030
:103395005CE07006900050E060028006756A0502E8
:1033A500327F75BB170238090238097E017F00E5B7
:1033B500BE123E16E5BD2FFF50010E8E578F589059
:1033C500005CE0B4017AE560455F6025AC5FAD6007
:1033D5001DBDFF011C8F028E038C068D079038C71B
:1033E50012002EE493FE740193FFEFC39AEE9B4007
:1033F500028005785F123E40AE5FAF6074B3BE00D9
:1034050021D39F401DAC57AD580FBF00010E90381A
:10341500C712002EE493FE740193FFEDC39FEC9E4B
:1034250040028005785F12003FAE5FAF6090005E9E
:10343500E0123E1674648E048F05FF123DF88D3C34
:10344500E56DB40129AE57AF58EFD39400EE94085B
:10345500400F900050E0B40104C2058002D20580FF
:103465000D900050E0B40104D2058002C20575BB81
:10347500160238090238097E017F00E5BE123E16A4
:10348500E5BD2FFF50010E8E578F5890005CE0B4BC
:10349500027AE560455F6025AC5FAD601DBDFF014B
:1034A5001C8F028E038C068D07903A3112002EE494
:1034B50093FE740193FFEFC39AEE9B40028005785B
:1034C5005F123E40AE5FAF6074B3BE0021D39F4034
:1034D5001DAC57AD580FBF00010E903A3112002EAA
:1034E500E493FE740193FFEDC39FEC9E40028005BB
:1034F500785F12003FAE5FAF6090005EE0123E164F
:1035050074648E048F05FF123DF88D3CE56DB402A1
:1035150029AE57AF58EFD39400EE9408400F9000B2
:1035250050E0B40104C2058002D205800D90005020
:10353500E0B40104D2058002C20590005CE070038E
:10354500753C00900050E07002C20575BB1F023843
:10355500090238097E017F00E5BE123E16E5BD2F42
:10356500FF50010E8E578F587409123E1674E68E61
:10357500048F05FF123DF88C388D39E56B2DFD5014
:10358500010C74018C068D07123E088E388F398523
:10359500396B75BB190238090238097E017F00E5D0
:1035A500BE123E16E5BD2FFF50010E8E578F587483
:1035B50004123E088F3F90006AE0B40102800302C6
:1035C5003676756300756300E563D394074003029F
:1035D500366CE56390002B123E2EE0D3953F501AD2
:1035E500E56390002B123E2EE0F404253FFEE563D3
:1035F50090087D123E2EEEF08017E56390002B12A9
:103605003E2EE0C3953FFEE56390087D123E2EEE0B
:10361500F0E563C39404400990006EE0C3956350E0
:103625003BE5636029E56390087D123E2EFEE0FFD1
:10363500EE900885E0D39F4013E56390087D123E28
:103645002EE0900885F0E563900886F0800E9008DE
:103655007DE0900885F07400900886F07863740129
:1036650026F640030235CD900886E0F4042408F5DB
:103675004790006AE0D394014033E53FD3946E4010
:1036850004D20C8002C20C75470590006AE0B402B2
:1036950005A20CB34002800375470790006AE0B4A9
:1036A5000306A20CB3B340028003754707E56C65BA
:1036B500476008E54304F54485476CE547B40708CA
:1036C500E5B54480F5B58006E5B5547FF5B5E54724
:1036D50064066005E547B40808E5B54410F5B5800E
:1036E50006E5B554EFF5B575BB130238090238097F
:1036F5007E017F00E5BE123E16E5BD2FFF50010E8F
:103705008E578F587404123E088F6990006BE0B491
:1037150002028003023804756300756300E563D314
:10372500940340030237B1E563900027123E2EE073
:10373500D39569501AE563900027123E2EE0F404F4
:103745002569FEE563900887123E2EEEF08017E5A9
:1037550063900027123E2EE0C39569FEE56390084D
:1037650087123E2EEEF0E5636029E5639008871227
:103775003E2EFEE0FFEE90088BE0D39F4013E563FD
:10378500900887123E2EE090088BF0E56390088C38
:10379500F0800E900887E090088BF0740090088CFC
:1037A500F07863740126F6400302372290006CE03E
:1037B500704DE52945286036E548C39403500A90C5
:1037C500088CE004C394034002800790088CE00451
:1037D500F548E548D39402400A90088CE004D39458
:1037E500025002800790088CE004F548801190088B
:1037F5008CE004F548E548D3940440037548017509
:04380500BB1880006C
:1038550002328802328B0233AD0233B00234790270
:10386500347C02355602355902359D0235A00236A3
:07387500F20236F5023809EA
:10380900E56A75F00284AFF07E00EF4E7002D2ECEB
:03381900056A221B
:093E2E002582F582500205832271
:10002E00EF2F500205832582F582E5833E2EF58360
:01003E00229F
:08000300C3EF9DFFEE9CFE22FD
:08003F000806B60002180622B3
:0D000E00A3E004F07006123E24E004F0228E
:083E40000816B6FF0218162255
:0E3E0800048007C3CE13CECF13CFD5E0F62231
:103C4600BC000FBE0008ED8FF084FFADF022E4FE4D
:103C5600FF22BE000DEF60FE54F0606F20E7030206
:103C66003CFCEAC0E0EBC0E078017A0075F001EEBA
:103C760020E710EF25E0FFEE33FE0AC5F023C5F07E
:103C860030E7F0EA5407F9096A7A007B0060010818
:103C9600C3EC9E40167004ED9F4010ED9FFDEC9E18
:103CA600FCE5F0CA4ACA03F5F08005E5F003F5F035
:103CB600C3EE13FEEF13FFD9D77908CACBCAD8D003
:103CC600EAFEEBFFD0E0FBD0E0FA22EC8FF084FCBA
:103CD600ED54F045F0C48FF084FEEDC454F045F089
:103CE600C48FF084FDEEC4FE54F02DFFEE540F3C5D
:103CF600FEADF07C0022790078008FF0EC7E082083
:103D0600E70DC3CD33CD33C933C9C833C8DEF0841C
:103D160049F9E5F08FF0BE00E6FD7C00E9FFE8FE1C
:013D2600227A
:0E3E1600F88FF0A4FFE5F0CE88F0A42EFE2277
:103DE800600D782B023DF2007830D8FED5E0F8223D
:103DF800EEC0E07E00123C46EFFDEEFCD0E0FE2275
:03000B00023D971C
:03001B00023DB2F1
:03002B00023DCDC6
:03000000023E3786
:093E370075816E75D0000209923C
:0B001E00E5822FF582E5833EF583228A
:0A3E24000582D58202158315822263
:103D9700C0E0C0F0C083C082C0D075D000120987D0
:103DA700D0D0D082D083D0F0D0E032C0E0C0F0C015
:103DB70083C082C0D075D00012098AD0D0D082D0FB
:103DC70083D0F0D0E032C0E0C0F0C083C082C0D062
:103DD70075D00012098DD0D0D082D083D0F0D0E03A
:013DE70032A9
:00000001FF
